:107E000001C0DDC0112484B7882361F083FF03C063
:107E100094B7947F94BF982F937021F4282E80E01C
:107E2000B9D0EEC085E08093810082E08093C000ED
:107E300088E18093C10086E08093C20089E180934D
:107E4000C4008FE0A7D0549A86E028E13EEF91E08D
:107E5000309385002093840096BBB09BFECF4C9A54
:107E6000A8954091C00047FD02C0815089F7EE24DB
:107E7000E39495E0D92E21E1C22E80D0C82F89E26B
:107E800089D0C13461F47AD0C82F8AD0C238E9F0E1
:107E9000C13811F488E001C083E069D065C0C23404
:107EA00011F484E103C0C53419F485E081D05CC0CD
:107EB000C53539F463D0082F61D0182F000F111F7A
:107EC00052C0C63521F484E073D080E0E6CFC436DA
:107ED00009F02CC053D052D0F82E50D0B82EC0E0AC
:107EE000D1E04CD08993FC12FCCF5AD0E5E4BE120D
:107EF00001C0FFCF83E0F80187BFE89507B600FC1B
:107F0000FDCFA0E0B1E0F8018D919D910C01E7BE9D
:107F1000E89511243296FA12F7CFF801D7BEE8950A
:107F200007B600FCFDCFC7BEE8951EC0C43771F48C
:107F300025D024D0F82E22D033D0E801FE0185913F
:107F4000EF0115D0FA94F110F9CF0EC0C53739F40E
:107F500027D08EE10CD085E90AD08FE09ECFC135C5
:107F600011F488E017D01CD080E101D086CF909129
:107F7000C00095FFFCCF8093C60008958091C0009B
:107F800087FFFCCF8091C00084FD01C0A89580913F
:107F9000C6000895E0E6F0E098E1908380830895BC
:107FA000EDDF803219F088E0F5DFFFCF84E1DFCF2D
:107FB000CF93C82FE3DFC150E9F7CF91F1CFFC0198
:107FC0000A0167BFE895112407B600FCFDCF667073
:0E7FD00029F0452B19F481E187BFE89508954B
:027FFE00000879
:0400000300007E007B
:00000001FF
